:1000000002093D120DB17F01020DA4020B1BBB01C1
:100010000689828A83E0225002E722BBFE02E322A5
:1000200089828A83E49322BB010CE58229F582E56B
:10003000833AF583E0225006E92582F8E622BBFEEA
:1000400006E92582F8E222E58229F582E5833AF580
:1000500083E49322BB010689828A83F0225002F74F
:1000600022BBFE01F322F8BB010DE58229F582E5F2
:10007000833AF583E8F0225006E92582C8F622BBD0
:10008000FE05E92582C8F222BB010A89828A83E043
:10009000F5F0A3E022500687F009E71922BBFE071E
:1000A000E3F5F009E3192289828A83E493F5F07479
:1000B000019322BB010A89828A83F0E5F0A3F02232
:1000C0005006F709A7F01922BBFE06F3E5F009F385
:1000D000192275F008758200EF2FFFEE33FECD3345
:1000E000CDCC33CCC58233C5829BED9AEC99E582A9
:1000F00098400CF582EE9BFEED9AFDEC99FC0FD535
:10010000F0D6E4CEFBE4CDFAE4CCF9A88222B80024
:10011000C1B90059BA002DEC8BF084CFCECDFCE5EF
:10012000F0CBF97818EF2FFFEE33FEED33FDEC3313
:10013000FCEB33FB10D703994004EB99FB0FD8E598
:10014000E4F9FA227818EF2FFFEE33FEED33FDECE1
:1001500033FCC933C910D7059BE99A4007EC9BFCD7
:10016000E99AF90FD8E0E4C9FAE4CCFB2275F01063
:10017000EF2FFFEE33FEED33FDCC33CCC833C81088
:10018000D7079BEC9AE899400AED9BFDEC9AFCE8B6
:1001900099F80FD5F0DAE4CDFBE4CCFAE4C8F92203
:1001A000EB9FF5F0EA9E42F0E99D42F0EC6480C8D6
:1001B00064809845F022EB9FF5F0EA9E42F0E99DBD
:1001C00042F0E89C45F022BB010789828A83020342
:1001D000A15005E9F8020255BBFE05E9F80203AD9E
:1001E00089828A830203B9BB010789828A8302025A
:1001F0009D5005E9F8020291BBFE05E9F80204747E
:1002000022BB010DE58229F582E5833AF5830202DE
:100210009D5007E92582F8020291BBFE07E925827D
:10022000F802047422BB010DE58229F582E5833AC8
:10023000F5830204285007E92582F8020408BBFE72
:1002400007E92582F802045DE58229F582E5833A13
:10025000F5830203B9E6FC08E6FD08E6FE08E6FFC2
:1002600022BB010DE58229F582E5833AF58302037D
:10027000D65007E92582F80203C9BBFE07E92582AB
:10028000F80203E2E58229F582E5833AF583020369
:10029000EFECF608EDF608EEF608EFF622ECF0A328
:1002A000EDF0A3EEF0A3EFF022A8828583F0D083D7
:1002B000D0821202C01202C01202C01202C0E47345
:1002C000E493A3C583C5F0C583C8C582C8F0A3C5A0
:1002D00083C5F0C583C8C582C822A42582F582E5FE
:1002E000F03583F58322BB010DE58229F582E58394
:1002F0003AF5830204925007E92582F8020480BB94
:10030000FE07E92582F80204A4E58229F582E58347
:100310003AF5830204B6BB0120E58229F582E58324
:100320003AF583D0F0D0E0F8D0E0F9D0E0FAD0E0B0
:10033000FBE8C0E0C0F002049B5018E92582F8D029
:1003400083D082D0E0F9D0E0FAD0E0FBC082C08355
:10035000020489BBFE18E92582F8D083D082D0E060
:10036000F9D0E0FAD0E0FBC082C0830204AD228A5B
:10037000838982E473EF4E6012EF60010EEDBB01E2
:100380000B89828A83F0A3DFFCDEFA2289F0500712
:10039000F709DFFCA9F022BBFEFCF309DFFCA9F0A2
:1003A00022E0FCA3E0FDA3E0FEA3E0FF22E2FC08C4
:1003B000E2FD08E2FE08E2FF22E493FC740193FDF3
:1003C000740293FE740393FF22E6FB08E6F908E645
:1003D000FA08E6CBF822E0F8A3E0F9A3E0FAA3E0FC
:1003E000FB22E2FB08E2F908E2FA08E2CBF822E499
:1003F00093F8740193F9740293FA740393FB2274D3
:1004000001FF3395E0FEFDFC080808E62FFFF61813
:10041000E63EFEF618E63DFDF618E63CFCF62274D4
:1004200001FF3395E0FEFDFCA3A3A3E02FFFF0E561
:1004300082158270021583E03EFEF0E5821582701F
:10044000021583E03DFDF0E582158270021583E020
:100450003CFCF0227401FF3395E0FEFDFC08080827
:10046000E22FFFF218E23EFEF218E23DFDF218E242
:100470003CFCF222ECF208EDF208EEF208EFF22278
:10048000E6FB08E6FA08E6F922EBF608EAF608E9E0
:10049000F622E0FBA3E0FAA3E0F922EBF0A3EAF0F6
:1004A000A3E9F022E2FB08E2FA08E2F922EBF20803
:1004B000EAF208E9F222E493FB740193FA740293DE
:1004C000F9228B088A09890A00750B01750C0075E1
:1004D0000D00E4F50EAB0BAA0CA90D75F014E50E9A
:1004E000A4F58285F0831200277003020684E50ECE
:1004F00075F014A429F9EA35F0FA90000A7FFF7E1E
:10050000FF7DFF7CFF120225E4FBFAF9F8C312011C
:10051000A05003020684E50E75F014A4FFAEF0AB04
:100520000B250DF9E50C3EFA90000412002714602B
:10053000541470030205CC2402600302066FAB0B57
:10054000AA0CA90D75F014E50EA4F58285F083E4DC
:10055000120066E92FF9EA3EFA9000011202E6E97C
:100560004A4B7003020684E50E75F014A4AB0B250C
:100570000DF9E50C35F0FA9000011202E674FF1255
:100580000054020684AB0BAA0CA90D75F014E50EFD
:10059000A4F58285F083E4120066E50E75F014A4DC
:1005A00029F9EA35F0FA9000011202E6E94A4B60B7
:1005B0001BE50E75F014A4AB0B250DF9E50C35F019
:1005C000FA9000011202E674FF120054E50E75F075
:1005D00014A4AB0B250DF9E50C35F0FAE9240AF962
:1005E000E43AFAC003C002C0011201C7C006C00746
:1005F000E50E75F014A4250DF9E50C35F0FA900020
:1006000006120261D007D006EF2BFFEE3AFEED395D
:10061000FDEC38FCD001D002D0031201E7E50E75E5
:10062000F014A4FFAEF0AB0B250DF9E50C3EFA90EB
:10063000000E1202E6E94A4B604AAB0BE50D2FF9BA
:10064000E50C3EFA9000111202E6C003C002C001A0
:10065000AB0BE50D2FF9E50C3EFA90000E1202E609
:1006600089828A83D001D002D0031203738015AB34
:100670000BAA0CA90D75F014E50EA4F58285F08384
:10068000E4120066050EE50EC3940550030204D57E
:100690007F00227828E67005120D6A80F6E4F508DE
:1006A000F509F509E50975F011A42464F582E4342F
:1006B00000F583E07004000207E4E50975F011A479
:1006C0002468F582E43400F583C083C082E0FCA393
:1006D000E0FDA3E0FEA3E0FFC0077828E6FBD0071B
:1006E000C3EF9BFFEE9400FEED9400FDEC9400FC44
:1006F000D082D08312029DE50975F011A42468F51B
:1007000082E43400F583E0FCA3E0FDA3E0FEA3E077
:10071000FFE4FBFAF9F8C31201A050030207E4E575
:100720000975F011A42468F582E43400F583C083D0
:10073000C082E0FCA3E0FDA3E0FEA3E0FFE50975B5
:10074000F011A4246CF582E43400F583E0F8A3E012
:10075000F9A3E0FAA3E0FBEF2BFFEE3AFEED39FD43
:10076000EC38FCD082D08312029DE50975F011A40B
:100770002465F582E43400F583E07011E50975F035
:1007800011A42464F582E43400F583E4F0E50975EE
:10079000F011A42470F582E43400F583E0FBA3E0BB
:1007A000FAA3E04A4B603CE50975F011A42473F903
:1007B000740035F0750A01F50B890C00AB0AFAC01C
:1007C00002E50975F011A42470F582E43400F58384
:1007D000A3E0FAA3E0F5828A83D0021203738F08A4
:1007E000008001000509E509C3940350030206A433
:1007F000E47828F60206938F1690009F7401F0A308
:100800007400F0A37400F0E4F52190009FE0FBA3D6
:10081000E0FAA3E0F975F014E521A4F58285F083F0
:10082000120027600302092FE51624FD501F8000E7
:1008300090009FE0FBA3E0FAA3E0F975F014E52136
:10084000A4F58285F083E41200667FFF22AF1AAE22
:1008500019AD18AC17C006C007E52175F014A4FF48
:1008600090009FE0FBA3E0FAA3E02FF9EA35F0FA4D
:10087000900006D007D006120201AF1AAE19AD18CB
:10088000AC17C006C007E52175F014A4FF90009FC7
:10089000E0FBA3E0FAA3E02FF9EA35F0FA90000AB2
:1008A000D007D006120201AB1BAA1CA91DC003C0B1
:1008B00002C001E52175F014A4FFAEF090009FE0A6
:1008C000FBA3E0FAA3E02FF9EA3EFA90000E120330
:1008D0001690009FE0FBA3E0FAA3E02FF9EA3EFAAE
:1008E000900004E51612006690009FE0FBA3E0FA7A
:1008F000A3E0F975F014E521A4F58285F083740175
:10090000120066AB1EAA1FA920C003C002C001E5E9
:100910002175F014A4FF90009FE0FBA3E0FAA3E090
:100920002FF9EA35F0FA900011120316AF212205D3
:1009300021E5216405600302080A7FFF2278FFE4B5
:10094000F6D8FD9000007F007E01E4F0A3DFFCDE1E
:10095000FA75812C020992020D88E493A3F8E493BE
:10096000A34003F68001F208DFF48029E493A3F8A2
:100970005407240CC8C333C4540F4420C883400414
:10098000F456800146F6DFE4800B010204081020D3
:100990004080900B69E47E019360BCA3FF543F301C
:1009A000E509541FFEE493A360010ECF54C025E077
:1009B00060A840B8E493A3FAE493A3F8E493A3C82F
:1009C000C582C8CAC583CAF0A3C8C582C8CAC583C0
:1009D000CADFE9DEE780BE8B088A09890A00750B49
:1009E00001120088FFE5F0706DEF24C4602824FB3D
:1009F0006053244170607B017A0079977F647E00A8
:100A00007D007C00120CEDD290AB08AA09A90AE483
:100A100075F03C1200B37B017A007997120BB6EFA8
:100A20007002FF22007B017A0079977F847E037D2C
:100A3000007C00120CEDC290AB08AA09A90AE4756B
:100A4000F0411200B37B017A007997120BB6EF7078
:100A500002FF220080A0E4F50BAB08AA09A90AF561
:100A6000F01200B37F0322EF701CEB7006EDF4521E
:100A70009A529BBB0107EDF4529AED429BEB640244
:100A80007043ED429A22EF6401701CEB7006EDF4A6
:100A900052915292BB0107EDF45291ED4292EB64F8
:100AA000027022ED429122EF64027019EB7006EDA4
:100AB000F452A152A2BB0107EDF452A1ED42A2BB38
:100AC0000203ED42A122120C4D120C99E4750FE8BD
:100AD000750E03F50DF50C7510FF75110D751205EA
:100AE000F513751400751524FB7A0079257D011224
:100AF0000BEAE4750FD0750E07F50DF50C7510FFB8
:100B000075110D75121BF513751400751524FB7AFC
:100B10000079257D02120BEAD2AF22C0E0C0F0C0FE
:100B200083C082C0D075D000C000C001C002C00325
:100B3000C004C005C006C007AF8AEF2418FFE43424
:100B4000FCFEC28DAD07EDF58A8E8C120CD2D0075B
:100B5000D006D005D004D003D002D001D000D0D030
:100B6000D082D083D0F0D0E0326033006401010045
:100B7000000000000100000001FF04C200000101AC
:100B800001000000006400000064FF09D7000001BC
:100B90000102000000006400000064FF0C7300000C
:100BA00001280004290000000001220001230001A7
:100BB00025FF0124FF008B0C8A0D890E120DAC8ECF
:100BC0000F8F10AB0CAA0DA90E1201C7C3E5109F21
:100BD000FFE50F9EFE900004120261E4FCFDD312BB
:100BE00001B67F0050027F0100228B088A09890A22
:100BF000AF05850F1A850E19850D18850C17851000
:100C00001B85111C85121D85131E85141F8515203B
:100C10001207F7AB08AA09A90AEF020054120D3116
:100C20007B027D017F01120A677B027D807F0212B9
:100C30000A677B027D407F02120A677B027D207F6C
:100C400002120A677B027D107F02020A677E007F24
:100C5000647D007B017A007900120375E4FFEF7573
:100C6000F014A42400F582E43400F583E4F00FBF0F
:100C700005EC228B088A09890A750B01120088701D
:100C800007E5F07003120DB5E4F50BAB08AA09A94E
:100C90000AF5F01200B37F0322120D457D01E4FF37
:100CA000120CB67F187EFC120D7BE4FD7F01120D45
:100CB000587F01020D9BEF7005538EFE8006BF0129
:100CC00003438E01BD01045389FB22BD0203438906
:100CD00004227829120255EF2401FFE43EFEE43D90
:100CE000FDE43CFC7829120291782806228B0C8ABC
:100CF0000D890E900004120201120DACAB0CAA0D6E
:100D0000A90E0201E78B088A09890AE5227004D23C
:100D1000A78002C2A70522532201228B088A0989D3
:100D20000AE5236004D2A68002C2A605235323014C
:100D300022E4F59AF591F5A1F59BF592F5A2F5A0BF
:100D4000F590F580225389F05388CD538EFEE4F55B
:100D50008CF58AC2A9C2B922EF7004C2A98002D25E
:100D6000A9ED7003C2B922D2B92200000000000030
:100D700000000000000000000000225389FC4389AD
:100D800001AD078D8A8E8C22120D92120693E4FE1D
:100D9000FF22120003120C1D020AC6EF7003C28C60
:100DA00022D28C22E5CF54F84FF5CF2278290202C7
:090DB00055E4F5CF2243CF1022D7
:00000001FF
